:020000040000FA
:020000002B28AB
:040002000034003492
:08000800FE000308FF000C18C4
:100010000A282628831203130C10F0308F000030BA
:100020008E0020192B21A50A08302506031D26283D
:10003000A501A60A3C302606031D2628A601A70A0C
:1000400006302706031D26280130A7007F088300FD
:10005000FE0E7E0E09008316031300308600860113
:10006000FF308500831203130730920007309F0092
:1000700000308E00F0308F00831603130C148312AF
:1000800003131014901490150B178B173E30A40017
:1000900087210230A8000508AA00AA0C2A0CFF3A02
:1000A0000739AA00A5018601A6010130A7002A0A86
:1000B000013A031973282A08013A03197C282A08EF
:1000C000023A031988282A08033A03199A282A08A9
:1000D000043A0319AC282A08053A0319BE282A084D
:1000E000063A0319D028640001302706031D7A2838
:1000F000861673288612732864002708013A031DA8
:100100007C280130A900D7206400201984287C288D
:100110000230A900D720640020198B28640027082A
:10012000023A031D8E280230A900D720640020194E
:1001300096288E280330A900D720640020199D2816
:1001400064002708033A031DA0280330A900D72024
:1001500064002019A828A0280430A900D720640032
:100160002019AF2864002708043A031DB228043080
:10017000A900D72064002019BA28B2280530A900A8
:10018000D72064002019C12864002708053A031D00
:10019000C4280530A900D72064002019CC28C42821
:1001A0000630A900D72064002019D328D028A00148
:0C01B000A201A217A101201506160800EC
:100200008207EE341D34DC3420340034FF3482079E
:10021000EE341D34DC3428340034FF348207EE34ED
:100220001D34DC342A340034FF348207EE341D34AC
:10023000DC342A3480340034FF348207EE341D3439
:10024000DC342A34A0340034FF348207EE341D3409
:10025000DC340034FF34A21F70292908013A031945
:1002600046292908023A03194B292908033A031998
:1002700050292908043A031955292908053A031970
:100280005A292908063A03195F295F2901308A0093
:1002900021080021632901308A00210807216329F0
:1002A00001308A0021080E21632901308A002108CB
:1002B0001521632901308A0021081D21632901309D
:1002C0008A0021082521A300A10AFF3C03197C29EB
:1002D000A31BA014A31FA010A30D0310A20C792927
:1002E000A31BA014A31FA010A30D0310A20C03189E
:1002F000A20CA01C83297F292011061208000C30B3
:1003000097008616080097018611861208002408B7
:10031000831603139200031083120313240C950019
:020320000800D3
:02400E00143F5D
:00000001FF
